:100000000429AD0001300428A6002E082C02031D8F
:100010000B282D082B02043003180130031902307D
:100020002605031D0130FF288030A100FE30A420EA
:100030000130A4207530AC003030CF28A101A117C9
:10004000B400FE30A4203408A428A501AF00B001FC
:10005000A01125080319A0150530A4002730AE0013
:1000600010303E200330AE00E8303E20AE01643058
:100070003E20AE010A303E202F084528AD00300852
:10008000AC002F08AB00E3202B08AB00A40303193E
:10009000A011250803194F282402031856282B08FD
:1000A000031DA011A0195628303EA4280800B20054
:1000B000061186118316061186110F3086058312EC
:1000C0003208A01881283E30AC008030CF20333079
:1000D000B10095201330AC008830CF2095206430DB
:1000E000CE2095206430CE202230B10095202830DB
:1000F00080200C30802006308020A0143208812817
:100100002014B100201C8F288611033C031C942866
:1001100094200530AC00DC30CF20031408002014FC
:10012000FE3C0319A2288615201C201006150F304E
:1001300086053108F03986040611B10E201895287D
:100140003230CE203208FF28A11B572883169B008F
:1001500083161C141A089B0AFF2883169A001C1584
:1001600055309D00AA309D009C149C18B5281C1188
:100170009B0AFF2883178001840AFF3E031DBB28CA
:10018000FF28AE01AD00FF30AD07031CAE07031C16
:10019000FF280330AC00DF30CF20C328AC01E83E9D
:1001A000AB00AC09FC30031CD828AB070318D528DA
:1001B000AB070000AC0FD5282B18DE28AB1CE228BB
:1001C0000000E2280800B001AF011030B1002C0D92
:1001D000AF0DB00D2D08AF022E08031C2E0FB0027C
:1001E0000318F9282D08AF072E0803182E0FB007A3
:1001F0000310AB0DAC0DB10BE7282B08FF288313C0
:100200008312031300000800A00107309F0083162B
:10021000FF308500FC30860081178312850186013E
:10022000203084006030BB20A03084005030BB20E0
:10023000203084003030BA200130AE00F430C220CB
:100240008614851A6A293C151420543057204530ED
:10025000572053305720543057204D3057204F30BF
:10026000572044305720453057202C30572020301D
:10027000572075305720203057206B30572075306D
:1002800057206E305720743057208030A100C03086
:100290001E20743057206F3057206530572074303F
:1002A000572073305720203057206C3057206F3044
:1002B000572073305720203057206C305720613042
:1002C000572074305720653057206E305720851ADC
:1002D0006A29672914204E305720753057206D3019
:1002E0005720572065305720723057206D305720E7
:1002F000653057206C3057206430572065305720C8
:100300007230572020305720563057202D3057203C
:10031000313057208030A100C0301E207730572068
:10032000572057202E3057207030572069305720E3
:100330006330572062305720613057207330572088
:1003400069305720633057202E3057206E305720A9
:100350006C3057200730AE00D030C2200130A620CC
:10036000A7002708031DB6293C15792D0301A620F7
:10037000D6000130A620D9000330DB000230A620D1
:10038000A700A7080319C52906140230590203184B
:10039000CB29CD21CC29E621122C1420473057201F
:1003A0006530572057206E305720203057206E3050
:1003B0005720753057206D30572057206530572013
:1003C00072305720733057203822080014204130F3
:1003D0005720613057206E305720773057206530D6
:1003E00057207A3057206930572067305720203007
:1003F00057208030A100A501FF305907AF00FF3022
:100400000318013EB0002820203057206E305720BE
:100410007230572003305902031C122A273057200C
:10042000733057200618372A8030A100C0301E20B4
:10043000473057206530572057206E3057202030E6
:1004400057206E305720693057206530572075305F
:1004500057207730572065305720203057206E3096
:10046000572072305720273057207330572008000C
:100470003C1D462A8030A100CC301E20543057202D
:100480004530572053305720543057200800D801AA
:100490008030A100C0301E204730572065305720E3
:1004A0006830572065305720753057206730572007
:1004B000653057206E305720203057207630572037
:1004C0006F3057206C305720051E672A642A851E1E
:1004D0007E2ADC0A0430C120FB305C02031C7A2A2D
:1004E0000230860683168610831286180614861C30
:1004F0000610DC01051E7D2A552B672A0614122CD6
:10050000023058020318852A122C06140230831672
:100510009B0001308312AD200330D700DA01FF3099
:100520005907A700FF300318013EA8002808031D43
:100530009D2A27085A020318D62A3C14DA0ADC013D
:10054000DC0A5C083D3E84000008A7005708A6208E
:10055000A9000F302905AA01A9002A08031DB42A01
:10056000290827020319B52A3C10D70A5708A620E4
:10057000A700F0302705A801A7002808AC0027082D
:10058000AB00AE0103010120BB0003305C0203019C
:10059000031801303B050319A02A58085C0203190F
:1005A000D22A3C103C1CD52AD62A8F2A3C18232B51
:1005B000560A83169B00F0308312AD200130DC0018
:1005C000B801F030B7005608A620A7002708B705E5
:1005D000B801BA010F30B9005C083D3E8400000844
:1005E000A9002908B905BA0137083904DD00560801
:1005F00083169B0083125D08AD20DC0A7B30560217
:100600000318042BD60A052B472A5C085802031846
:10061000E02AD90A560883169B008312590EB700A8
:10062000B800F030B7050F30B8053708AD203808EE
:10063000AD2083169B0183125608AD205908AD20CA
:100640000130AD204E2B0330D7005708A620DC0028
:10065000D70AA8015C0E0F39A7002808031D252B17
:1006600027085A02031D252B5708A620A700F030A3
:100670002704DC00570883169B0083125C08AD201A
:100680000130DC00013086068316061064308312C8
:10069000C120DC0A29305C02031C422B051E512BB1
:1006A0004E2B3230C1203C10122C0130C1200301EE
:1006B00005180130B801B700BA010230B900390895
:1006C000851C0301B9003A08851C0301BA003908EA
:1006D000B7073A080318013EB807BA010430B90059
:1006E0003908051D0301B9003A08051D0301BA00C8
:1006F0003908B7073A080318013EB807BA010830AD
:10070000B9003908851D0301B9003A08851D0301A8
:10071000BA0037083907D5000B30550203190130EC
:10072000031D0301BB0003013C1901303B05BB0065
:10073000550803190130031D03013B040319AF2BB6
:1007400014204E305720723057203A30572038222C
:1007500083301E20A1018614BC140330DB00BC1CB6
:10076000E52B55080319B82B0B305502031DB92B87
:10077000E42B55080319D52B0B3055020318D52B44
:100780000A305502031DC52BD5018030A100550844
:100790002520D80A58083D3E8400550880000F30B7
:1007A0005802031CD42B802AE42B0C305502031D65
:1007B000DD2B3C1DDC2B802AE42B0F305502031D62
:1007C000E32B802AE42B122CE62B122C3A30D1009A
:1007D0009830D0000301051A0130BB005108AC006D
:1007E0005008AB00AE01030101203B050319FF2BAC
:1007F0006430CE20D003500A0319D103EA2B3A30DB
:10080000D1009830D000051A112C6430CE20D003CE
:10081000500A0319D10351085004031D102C802ADB
:10082000032C552B7530CF003030CE00BC10D801D2
:10083000DC015C083D3E840000308000DC0A1030A2
:100840005C02031C192C851A262C362C051E292C1B
:10085000552B4F084E04031D2F2C8610352C0130CC
:10086000C120CE034E0A0319CF03232C8614753002
:10087000CF003030CE0004305602031C1A2DD301B5
:10088000D201D20A0319D30A0A30C120061C4A2C0D
:10089000D301D201851E4D2C522C5208C83A530464
:1008A000031D412C5308031D592CC8305202031C50
:1008B0005A2C1B2D5B08A620D40014208030A100E8
:1008C000C0301E204E305720723057203A3057200B
:1008D000A501F0305405B801B7003708AF0038085B
:1008E000B0000430AB000310B00CAF0CAB0B732C9A
:1008F00028202F305720A501FF305907AF00FF30C7
:100900000318013EB00028205B0ADC005C08A6202A
:10091000A70010302702031CA12C203057202A30BA
:1009200057204E3057202A3057205C08A620A700B9
:100930000F302705DD005C0883169B0083125D08DD
:10094000AD20382280301E20A1018030A100A501F9
:100950000F305405B001AF002820DB0A5B08A62049
:10096000D40010305402031CA52CF0305405B801FB
:10097000B7003708A7003808A8000430AB00031000
:10098000A80CA70CAB0BBF2C2808031DCD2C2708E7
:100990005902031DCD2C0330DB00061CEE2C033066
:1009A000D7005708A620A700F0302705A801A70008
:1009B0002708F03A2804031DDE2CE32CD70A7B30ED
:1009C0005702031DD12C7B305702031DE82C061063
:1009D000023083169B0003018312AD20851AF12C8F
:1009E000EE2C0A30C120D301D201D20A0319D30A56
:1009F0000130C1204F084E04031D002D8610042D28
:100A0000CE034E0A0319CF03061C082DD301D201D1
:100A1000851A0B2D362C051E0E2D552B53083A3AF0
:100A2000983003195206031DF52C0618182DE621DF
:100A30000330DB00122C14204E3057207530572025
:100A40006D30572057206530572072305720733053
:100A50005720203057207730572069305720733087
:100A600057205720653057206E3057203F30572091
:100A70008030A100C0301E20543057204F30572006
:100A80004530572054305720533057203D305720A1
:100A90004230572065305720763057206530572038
:100AA00073305720743057206930572067305720F3
:100AB000653057206E3057203822851A602D5D2D05
:100AC0000A30C120C830DC000301851A0130BB00A8
:100AD00001305C020301031801303B050319742D3A
:100AE0001430C120DC03642D5C08031D792DE62140
:100AF000122C14204E305720753057206D3057205F
:100B000057206530572072305720733057202030DF
:100B10005720773057206F3057207230572064307D
:100B20005720653057206E3057208030A100C030EC
:100B30001E206730572065305720773057206930A6
:100B400057207330572074305720213057203822D7
:100B5000033083169B0010308312AD200430D60082
:100B6000560883169B0003018312AD20D60A7C3001
:100B70005602031CB02D0130DC00013086068316BE
:100B80000610C8308312C120DC0A0B305C02031C43
:100B9000BD2DCD210330D6000130D9000330DB005C
:100BA000061083169B0183125608AD205908AD200C
:100BB0000301AD20851ADD2DDA2D0A30C120122C5B
:02400E00103F61
:084200000300000000001000A3
:00000001FF
